:100000000C9479000C94DE010C9496000C949600EC
:100010000C9496000C9496000C9496000C94960008
:100020000C9496000C9496000C9496000C949600F8
:100030000C9496000C9496000C9496000C949600E8
:100040000C9496000C9496000C9496000C949600D8
:100050000C9496000C9496000C9496000C949600C8
:100060000C9496000C94960009022200010100A055
:100070000A09040000010300000009210101000138
:1000800022340007058103080064120110010000FA
:100090000008C016E8030001010200010C034D0036
:1000A0006F0075007300650012036F00620064004A
:1000B000650076002E006100740004030904050148
:1000C0000902A1010901A10005091901290315006F
:1000D00025019503750181029501750581030501CF
:1000E0000930093109381581257F75089503810686
:1000F000C0C011241FBECFEFD4E0DEBFCDBF11E0E2
:10010000A0E0B1E0E8E0F7E002C005900D92A43075
:10011000B107D9F721E0A4E0B1E001C01D92A234FB
:10012000B207E1F70E9420030C9482030C940000B4
:10013000CF93C62F2091170124FF19C020911801D9
:1001400038E82327209318012C2FFC01A9E1B1E006
:1001500081918D9321501216DCF36C2F89E191E08F
:100160000E94DA01CC5FC0931701CF9108952AE570
:1001700020931701E9CFCF93DF938091280183501B
:1001800087FD28C0909124019D3211F5883001F53A
:1001900080912501CCE0D0E0C81BD109C45DDE4FC1
:1001A00083EC80930C018AE5809301011092040195
:1001B0008881807609F45BC0CE010E94FF029F8196
:1001C000911104C09E81981708F4892F8093000133
:1001D000109228018091010184FF3CC080910001B0
:1001E0008F3FC1F1C82F893008F0C8E08C1B809385
:1001F000000180910C0198E8892780930C01CC23A1
:10020000E1F040912601509127018091040186FF81
:10021000A6C0ADE0B1E0FA019C2F84918D93319698
:100220009150D9F72FEF2C0F30E02F5F3F4F240F65
:10023000351F30932701209326016C2F8DE091E02C
:100240000E94DA01CC5FCC3019F08FEF809300016F
:10025000C093010184E199B1947131F48150D9F7CF
:100260001092290110922301DF91CF9108952A81E4
:1002700010921501998191110AC01092160125E181
:1002800031E082E0309327012093260198CF95300A
:1002900029F42093290125E131E0F4CF963009F0CB
:1002A00047C09B81913041F48AE890E09093270108
:1002B0008093260182E109C0923059F488E690E0EB
:1002C000909327018093260182E290E490930401A9
:1002D00076CF9330C9F4211108C08AEB90E0909357
:1002E00027018093260184E0F0CF213019F488EAB9
:1002F00090E0DCCF223049F78CE990E09093270121
:10030000809326018CE0E1CF913241F48AE790E0BE
:10031000909327018093260189E0D7CF9232A9F6E6
:100320008EEB90E0909327018093260184E3CDCF5C
:10033000983071F0993019F420932B01ACCF9A309A
:1003400059F09B3009F0A7CF9BE490931801A3CFFD
:100350002BE231E081E096CF25E131E0FBCFDA01FD
:10036000EDE0F1E09C2F8D9181939150E1F75ACF10
:10037000E9E6F0E0808182608083E89AE7E1F1E0DD
:100380008BE481838AE580830895A82FB92F80E0CC
:1003900090E041E050EA609530E009C02D9182275D
:1003A0009795879510F084279527305EC8F36F5F87
:1003B000A8F30895EADF8D939D930895CF93CFB767
:1003C000CF93DF93C3954C9BE9F74C9B0BC04C9BA1
:1003D00009C04C9B07C04C9B05C04C9B03C04C9B69
:1003E00001C08BC06F93C0912501DD27C45DDE4F36
:1003F0002F9365E54C9B03C02F916F91E6CF0F9330
:100400001F934F9320E040E15F9309B1047104FB17
:1004100027F93F9350E03BE039C0147140642F77D7
:10042000012F5F5F1EC0406819B114712F775250C1
:100430001FC0406409B12F770471D1F15F5F00C024
:1004400023C0406219B12F77147191F15F5F00C032
:1004500025C004711027515012F45D5F0000115047
:1004600027952C3F19B1C8F6147101270150279523
:100470002C3FC8F64227499309B1047110274F73E6
:10048000115027952C3FA8F64695469519B1147141
:1004900079F00127015027952C3F98F66B5A60F3AD
:1004A000315009B1B0F600C011E01CBB002719C0E3
:1004B0003B503195C31BD04011E01CBB0881033C6D
:1004C00009F10B34F9F0209123011981110F121356
:1004D000EDCF4A81441F093651F10D3211F0013E32
:1004E00029F700932A013F915F914F911F910F913E
:1004F0002F916F91CCB3C0FD65CFDF91CF91CFBF6E
:10050000CF91189520912A01222369F31091280197
:10051000112391F5343092F1309328012093240176
:10052000109125013BE0311B3093250127C000913C
:10053000280101300CF50AE54F7049F430910101B2
:1005400034FD1DC000930101CCE0D1E01CC030910E
:10055000170134FD14C000931701C8E1D1E013C0A6
:10056000052710E000C000000BB91AC0052710E0F5
:10057000221F1DC010E021C04AE502C032ED432F0A
:10058000C4E1D0E032E01AB114615C9A0BB11AB93F
:1005900054E120E865E320FF05270BB9279517955F
:1005A0001C3FF0F66695B8F7B1F720FF05270BB9A9
:1005B000279517951C3FD0F62795179517FF052708
:1005C00000001C3F0BB9B0F629913A9519F70B7E44
:1005D00010912901110FC651D0400BB911F01093A1
:1005E000230111E01CBB00611AB11B7E402F4B7E22
:1005F00054E05A95F1F70BB91AB94BB974CFFC0115
:10060000808180768032D1F48181813041F488E02C
:1006100091E0909327018093260184E00895823031
:1006200041F485E091E0909327018093260181E0D9
:1006300008958A3019F483818093050180E008953C
:100640009EE088E10FB6F894A895809360000FBEF5
:10065000909360000E94B801549A80E0815009F0A4
:1006600043C054987894A8950E94BB0080911701CC
:1006700084FFF9CF40910601509107011416150629
:10068000DCF120EE3FEF240F351F66E0359527950E
:100690006A95E1F72093090180910201909103018D
:1006A000820F911D27FD9A9590930301809302017B
:1006B0001816190624F120EE3FEF820F931F26E053
:1006C000959587952A95E1F780930A01481B510972
:1006D00087FD5395509307014093060164E088E03D
:1006E00091E00E949800BFCFA895EFE9FFE0319715
:1006F000F1F700C00000B2CF20E230E0C4CF20E22A
:0807000030E0DBCFF894FFCFDD
:04070800FF5AC001D3
:00000001FF
